:0500000002003361DF86
:02000B0061E0B2
:0200130081402A
:02001B00814121
:02002300814218
:02002B0081430F
:10003300759840758780758921758DFF758BFF7560
:100043008850D29975816075A8827530007531002A
:10005300753700753807D214D215D216D217D218B5
:10006300D219D21AD21BD21CD21DD21ED21FD22019
:10007300D221D222D223D224D225D226D227D228C9
:10008300D229D22AD22BD22CD22DD22ED22FD23475
:10009300D235D236D237D250C251C291D2922092A7
:1000A30014301421C214B215201505120452801500
:1000B30012045F801020140DD21420150512045B66
:1000C3008003120468D291D293209314301621C274
:1000D30016B21720170512046C80151204798010CC
:1000E30020160DD216201705120475800312048200
:1000F300D294209414301821C218B2192019051271
:1001030004868015120493801020180DD21820192C
:100113000512048F800312049CD295209514301A83
:1001230021C21AB21B201B051204A080151204ADB4
:100133008010201A0DD21A201B051204A980031265
:1001430004B6D296209614301C21C21CB21D201D69
:10015300051204BA80151204C78010201C0DD21C8E
:10016300201D051204C380031204D0D297209714D4
:10017300301E21C21EB21F201F051204D480151287
:1001830004E18010201E0DD21E201F051204DD8005
:10019300031204EAD2A020A014302021C220B221ED
:1001A3002021051204EE80151204FB801020200D7F
:1001B300D2202021051204F78003120504D2A120C6
:1001C300A114302221C222B2232023051205088064
:1001D30015120515801020220DD2222023051205A9
:1001E30011800312051ED2A220A214302421C2249E
:1001F300B225202505120522801512052F80102017
:10020300240DD22420250512052B8003120538D294
:10021300A320A314302621C226B2272027051205C6
:100223003C8015120549801020260DD22620270573
:100233001205458003120552D2A420A414302821AC
:10024300C228B2292029051205568015120563809C
:100253001020280DD22820290512055F80031205DE
:100263006CD2A520A514302A21C22AB22B202B053B
:10027300120570801512057D8010202A0DD22A20C8
:100283002B051205798003120586D2A620A6143009
:100293002C21C22CB22D202D0512058A80151205A2
:1002A300978010202C0DD22C202D0512059380034E
:1002B3001205A0D2A720A714302E21C22EB22F20C0
:1002C3002F051205A480151205B18010202E0DD222
:1002D3002E202F051205AD80031205BAD2B220B22B
:1002E30014303421C234B2352035051205BE8015D1
:1002F3001205E7801020340DD2342035051205E3B2
:10030300800312060CD2B320B314303621C236B2A6
:10031300372037051206108015120630801020365C
:100323000DD23620370512062C800312064CD2B4A8
:1003330020B41C753207120650120444D5320675D8
:10034300320112065012044BD2B420B40280EDD213
:10035300B520B51C75320712066B120444D532065C
:1003630075320112066B12044BD2B520B50280ED33
:10037300D2B620B61C753207120686120444D53253
:100383000675320112068612044BD2B620B60280DD
:10039300EDD2B720B71C7532071206A4120444D558
:1003A30032067532011206A412044BD2B720B702EB
:1003B30080EDE580F535A836A935C2D7E899400622
:1003C30024FE50108008C2D7E99824FE50068535D4
:1003D300361206C2438701019D02003332C0D0C0EA
:1003E300E0C083C082305010C250C2B0D2517533C6
:1003F30000753400D2908018205115B2900533E572
:10040300339006E393F58CD082D083D0E0D0D03202
:10041300B2900534E534B4FF10C251D290758CFF0D
:10042300D082D083D0E0D0D032B40A02D2B09007C9
:10043300E393F58CD082D083D0E0D0D03232323205
:10044300327E20DFFEDEFC227E60DFFEDEFC22D277
:10045300507537081204442212044422D2507537CF
:10046300081204442212044422D25075370912049C
:10047300442212044422D250753709120444221232
:10048300044422D250753807120444221204442231
:10049300D2507538071204442212044422D25075F4
:1004A300380A1204442212044422D25075380A1224
:1004B30004442212044422D25075385D12044422AB
:1004C30012044422D25075385D12044422120444AB
:1004D30022D25075385B1204442212044422D250B3
:1004E30075385B1204442212044422D2507537003B
:1004F3001204442212044422D250753700120444D9
:100503002212044422D250753701120444221204E9
:100513004422D2507537011204442212044422D2D9
:10052300507537021204442212044422D250753704
:10053300021204442212044422D2507537031204D7
:10054300442212044422D250753703120444221267
:10055300044422D250753704120444221204442264
:10056300D2507537041204442212044422D2507527
:1005730037051204442212044422D250753705125F
:1005830004442212044422D2507537061204442232
:1005930012044422D2507537061204442212044432
:1005A30022D2507537071204442212044422D25037
:1005B3007537071204442212044422D250E5300452
:1005C300B40801E4F5303099FDC299F539E53724D3
:1005D300C0F599E5393099FDC299F5991204442281
:1005E30012044422D250E53004B40801E4F530305B
:1005F30099FDC299F539E53724C0F599E539309964
:10060300FDC299F5991204442212044422D25030B7
:1006130099FDC299E53724C0F5993099FDC29975C2
:1006230099017530011204442212044422D250303D
:1006330099FDC299E53724C0F5993099FDC29975A2
:1006430099007530001204442212044422D250301F
:1006530099FDC299E53724C0F5993099FDC29905F2
:1006630031E531547FF59922D2503099FDC299E595
:100673003724C0F5993099FDC2991531E531547F7E
:10068300F59922D2503099FDC299E53724B0F599F6
:100693003099FDC2997599603099FDC29975990099
:1006A30022D2503099FDC299E53724B0F59930999B
:1006B300FDC2997599613099FDC29975990022D24D
:1006C300503099FDC299E53724B0F5993099FDC2B0
:1006D300998538993099FDC299E535C313F5992267
:1006E300FFE0FFE0FFE0FFE0FFE0FEE1FEE1FEE10F
:1006F300FEE1FEE1FDE2FDE2FDE2FDE2FDE2FCE3FF
:10070300FCE3FCE3FCE3FCE3FBE4FBE4FBE4FBE4EE
:10071300FBE4FAE5FAE5FAE5FAE5FAE5F9E6F9E6DE
:10072300F9E6F9E6F9E6F8E7F8E7F8E7F8E7F8E7CE
:10073300F7E8F7E8F7E8F7E8F7E8F6E9F6E9F6E9BE
:10074300F6E9F6E9F5EAF5EAF5EAF5EAF5EAF4EBAE
:10075300F4EBF4EBF4EBF4EBF3ECF3ECF3ECF3EC9E
:10076300F3ECF2EDF2EDF2EDF2EDF2EDF1EEF1EE8E
:10077300F1EEF1EEF1EEF0EFF0EFF0EFF0EFF0EF7E
:10078300F0EFF0EFF0EFF0EFF0EFF0EFF0EFF0EF6E
:10079300F0EFF0EFF0EFF0EFF0EFF0EFF0EFF0EF5E
:1007A300F0EFF0EFF1EEF1EEF2EDF2EDF3ECF3EC4E
:1007B300F4EBF4EBF5EAF5EAF6E9F6E9F7E8F7E83E
:1007C300F8E7F8E7F9E6F9E6FAE5FAE5FBE4FBE42E
:1007D300FCE3FCE3FDE2FDE2FEE1FEE1FFE0FFE01E
:1007E300E0FFE3FCE6F9E9F6ECF3EFF0F2EDF5EA0E
:1007F300F8E7FBE4FEE1FFE0FFE0FFE0FFE0FFE0FE
:10080300FEE1FEE1FEE1FEE1FEE1FDE2FDE2FDE2ED
:10081300FDE2FDE2FCE3FCE3FCE3FCE3FCE3FBE4DD
:10082300FBE4FBE4FBE4FBE4FAE5FAE5FAE5FAE5CD
:10083300FAE5F9E6F9E6F9E6F9E6F9E6F8E7F8E7BD
:10084300F8E7F8E7F8E7F7E8F7E8F7E8F7E8F7E8AD
:10085300F6E9F6E9F6E9F6E9F6E9F5EAF5EAF5EA9D
:10086300F5EAF5EAF4EBF4EBF4EBF4EBF4EBF3EC8D
:10087300F3ECF3ECF3ECF3ECF2EDF2EDF2EDF2ED7D
:10088300F2EDF1EEF1EEF1EEF1EEF1EEF0EFF0EF6D
:10089300F0EFF0EFF0EFF0EFF0EFF0EFF0EFF0EF5D
:1008A300F0EFF0EFF1EEF1EEF2EDF2EDF3ECF3EC4D
:1008B300F4EBF4EBF5EAF5EAF6E9F6E9F7E8F7E83D
:1008C300F8E7F8E7F9E6F9E6FAE5FAE5FBE4FBE42D
:1008D300FCE3FCE3FDE2FDE2FEE1FEE1FFE0FFE01D
:1008E300204D757A796B616E7420342076312E3009
:1008F3006720323030362D31322D323820286329AB
:100903004164616D20536D69616C656B206A616E32
:100913006B6F6D757A796B616E744077702E706C46
:10092300207777772E736D69616C656B2E707276A5
:100933002E706C2057737A656C6B696520707261D9
:100943007761207A617374727A657A6F6E652E208F
:100953004A616B69656B6F6C7769656B207A61734C
:10096300746F736F77616E6961206B6F6D6572630E
:10097300796A6E65206B6F6475206E6965646F7A42
:10098300776F6C6F6E652E20416C6C2052696768BF
:1009930074732052657365727665642E20467265A2
:1009A3006520666F72206E6F6E20636F6D6D65726A
:0B09B3006369616C206F6E6C792E2070
:00000001FF
